:100000000C9461010C9489010C9489010C94890170
:100010000C9489010C9489010C9489010C94890138
:100020000C9489010C9489010C9414150C9483157B
:100030000C9489010C9489010C9489010C94890118
:100040000C9489010C9489010C9489010C94890108
:100050000C9489010C9489010C9489010C94CA14A4
:100060000C9489010C9489010C9489010C948901E8
:100070000C9489010C9489010C9489010C948901D8
:100080000C9489010C9489010C9489010C948901C8
:100090000C9489010C9489010C9489010C948901B8
:1000A0000C9489010C94C5170C948901080B00026B
:1000B0000202000009040000010202000005240001
:1000C0001001052401010104240206052406000193
:1000D0000705810310004009040100020A00000026
:1000E00007050202400000070583024000000403E8
:1000F000090412010002EF02014041233680000191
:100100000102030141726475696E6F204C4C43001B
:100110004D482D4465766963652841726475696E42
:100120006F2900000000002300260029002C002F6A
:100130000000000000240027002A002D00300000ED
:10014000000000250028002B002E003100040404CC
:10015000040403040502020202040302020202066E
:10016000060606060604040202020404040802014C
:1001700010408040102040804080080204018040F0
:1001800020100201108010204040200000000200DA
:10019000090F0000030401000C0000000000000033
:1001A000000000000000000000000000000000004F
:1001B00000002A2B280000000000000000000000C2
:1001C000000000000000000000002C9EB4A0A1A2CE
:1001D000A434A6A7A5AE362D3738271E1F2021220E
:1001E00023242526B333B62EB7B89F848586878807
:1001F000898A8B8C8D8E8F909192939495969798F7
:10020000999A9B9C9D2F3130A3AD350405060708B4
:10021000090A0B0C0D0E0F101112131415161718D6
:10022000191A1B1C1DAFB1B0B50005010902A101CF
:100230000901A100850105091901290515002501FC
:10024000950575018102950175038103050109304A
:10025000093109381581257F750895038106050C3C
:100260000A38021581257F950175088106C0C005F1
:10027000010906A1018502050719E029E7150025F6
:100280000175019508810295017508810395067530
:1002900008150025FE0507190029FE8100C0050C80
:1002A0000901A10185041500250109E909EA09E20E
:1002B000750195038102750195058103C0004C18F5
:1002C000521F11241FBECFEFDAE0DEBFCDBF11E019
:1002D000A0E0B1E0EAE5F5E402C005900D92AE3C85
:1002E000B107D9F724E0AEECB1E001C01D92A23114
:1002F000B207E1F711E0C0E6D1E004C02197FE01AA
:100300000E948B20CF35D107C9F70E94C61B0C94E1
:10031000A0220C9400004F925F926F927F928F9276
:100320009F92AF92BF92CF92DF92EF92FF920F9384
:100330001F93CF93DF93E5010C151D052E053F0597
:100340000CF051C02801390146015701882309F4F6
:100350004FC0CA01DB0184159505A605B70514F445
:10036000D301C201B501A40188159905AA05BB05F1
:1003700014F4AC01BD01C016D106E206F30664F424
:10038000D501C401841B950BA60BB70BAC01BD01B5
:10039000440D551D661D771D9A01AB0124193509C1
:1003A00046095709AFEFBFEF0E940420A501940151
:1003B00024193509460957090E94E51F2883398306
:1003C00082E090E0DF91CF911F910F91FF90EF902D
:1003D000DF90CF90BF90AF909F908F907F906F9065
:1003E0005F904F9008952601370148015901AECF23
:1003F00090E080E0E7CF9091DE02911103C08FEF93
:100400009FEF08954FB7F89492E09093E900909190
:10041000F200292F30E01216130614F421E030E028
:10042000232B29F084E68093DD028091F10099234B
:1004300039F02091F200211103C02BE62093E8004F
:100440004FBF9923E1F290E0089581508F3008F07A
:1004500047C0E82FF0E0E15DFD4F0C948B204C028B
:1004600050023E02440248027002700270025302BF
:1004700059025D026102670270026B028091800086
:100480008F77809380000895809180008F7DF9CFD1
:1004900080918000877FF5CF84B58F7784BD0895E4
:1004A00084B58F7DFBCF809190008F7780939000F3
:1004B0000895809190008F7DF9CF80919000877F83
:1004C000F5CF8091C0008F778093C0000895809110
:1004D000C0008F7DF9CF8091C200877F8093C200DA
:1004E0000895CF93DF93282F30E0F901E557FE4FB1
:1004F0008491F901E459FE4FD491F901E35BFE4F79
:10050000C491CC2389F081110E942502EC2FF0E0E8
:10051000EE0FFF1FE15CFE4FA591B4918FB7F894E9
:10052000EC91DE2BDC938FBFDF91CF910895CF93B9
:10053000DF9390E0FC01E459FE4F2491835B9E4FD2
:10054000FC0184918823D1F090E0880F991FFC0171
:10055000EF5CFE4FA591B491FC01E15CFE4FC591AB
:10056000D491623071F49FB7F8943C91822F8095BA
:1005700083238C93E8812E2B28839FBFDF91CF911B
:1005800008958FB7F894EC912E2B2C938FBFF6CF54
:100590003FB7F8948091D9029091DA02A091DB02E2
:1005A000B091DC0226B5A89B05C02F3F19F001963B
:1005B000A11DB11D3FBFBA2FA92F982F8827BC01BD
:1005C000CD01620F711D811D911D42E0660F771FE5
:1005D000881F991F4A95D1F708958F929F92AF92E5
:1005E000BF92CF92DF92EF92FF926B017C010E944B
:1005F000C8024B015C01C114D104E104F104B9F05B
:100600000E94C802681979098A099B09683E7340EB
:100610008105910580F321E0C21AD108E108F108B3
:1006200088EE880E83E0981EA11CB11CE4CFFF90D9
:10063000EF90DF90CF90BF90AF909F908F900895F4
:1006400008954091A1025091A20220919F02309101
:10065000A00242175307B4F49091E8009570E1F3BB
:100660009091E80092FD19C08093F1008091A10261
:100670009091A20201968F739927892B19F48EEF1E
:100680008093E8008091A1029091A202019690933C
:10069000A2028093A10281E0089580E00895EF9284
:1006A000FF920F931F93CF93DF93F82E192FE62E0F
:1006B000042F81E0860F880F0E94210383E00E94AF
:1006C0002103CF2DD12FEC0EFD2EF11CCE15DF0511
:1006D000B9F007FF13C0FE0184910E942103182F77
:1006E00080E00E942103812321968111EFCFDF91C9
:1006F000CF911F910F91FF90EF9008958881EDCFDA
:1007000081E0F5CFDF92EF92FF920F931F93CF938B
:10071000DF93D82E8A01EB017B01E40EF51ECE1586
:10072000DF0559F0D7FE12C0FE0184910E9421031B
:1007300021968111F4CF0FEF1FEFC801DF91CF9108
:100740001F910F91FF90EF90DF9008958881EECF79
:100750002FB7F89487708093E9009091E800892F73
:10076000807295FF04C09091F20080E4891B2FBF36
:1007700008957F928F929F92AF92BF92CF92DF9215
:10078000EF92FF920F931F93CF93DF93C82E8B01AD
:100790007A018091DE02811110C08FEF9FEFDF910F
:1007A000CF911F910F91FF90EF90DF90CF90BF906E
:1007B000AF909F908F907F9008958091A50280FFC9
:1007C00005C08091E00082608093E000CE2DDF2D97
:1007D000D12C8AEFB82E8C2D8770982E8C2D80729C
:1007E000882E8C2D8074782E9AE3A92E209719F4E8
:1007F000DD2009F452C08C2D0E94A80381110AC08B
:10080000BA94BB2051F261E070E080E090E00E9479
:10081000ED02ECCF8C171D0611F00CF08C2F9FB75A
:10082000F8949092E9002091E80025FD02C09FBF56
:10083000DDCF282F30E0C21BD30B882029F0815058
:10084000A0F01092F100FBCFF801C7FC0AC0815064
:1008500050F041914093F100FACF44914093F10060
:1008600031968150D0F7020F131FDD2021F0A092A6
:10087000E800D12CDCCF8091E80085FD07C0A09274
:10088000E800DD24D394209791F2F3CF209779F6F6
:10089000772069F2A092E800CACF84E68093A40290
:1008A000C7017DCF8091970281110DC082E08093B6
:1008B000930284E080939402109296021092950223
:1008C00081E08093970283E992E008950F931F934C
:1008D000CF93DF931F92CDB7DEB782E0898342E4E6
:1008E00050E06CEA70E080E80E9482030E945204AB
:1008F000DC0112960D911C910115110589F0D801AA
:10090000ED91FC910280F381E02DBE016F5F7F4F7E
:10091000C801099597FD04C0F80100851185ECCF49
:1009200089810F90DF91CF911F910F910895CF93FF
:10093000DF93FC01DB01818114963C911497682FB1
:10094000630F7727771F683071059CF5C281D381CB
:10095000209739F5B383A283908112969C931297C6
:1009600013968C93139715968C911597890F808306
:1009700090E080E0831708F52181C22FD0E0BE010E
:100980006E5F7E4F16964D915C911797480F591FD9
:10099000EA014881EB0148832F5F21830196EACF6A
:1009A000EA014885598541155105D1F7B987A887CE
:1009B000D3CF80E0DF91CF91089581E0FBCFCF933B
:1009C000DF93EC0180911401882331F083E00E94D1
:1009D000B9031816190634F081E090E09B838A83EE
:1009E00080E090E0DF91CF910895FC014481558132
:1009F0006081718183EE92E00C94DF04CF93DF93EA
:100A00001F92CDB7DEB76983DC01ED91FC910280C6
:100A1000F381E02D41E050E0BE016F5F7F4F09950B
:100A20000F90DF91CF91089583E08093E90080914A
:100A3000F200882319F08AE38093E800089583E0A8
:100A40000E94A80390E00895FC018485958597FD98
:100A500005C02FEF3FEF3587248708950C94FB01E5
:100A60002FB7F8948091DF029091E002A091E1020B
:100A7000B091E2022FBF8093EB029093EC02A0931F
:100A8000ED02B093EE0283EE92E00E94240597FF00
:100A900026C02FB7F8948091DF029091E002A091D8
:100AA000E102B091E2022FBF4091EB025091EC02C3
:100AB0006091ED027091EE02841B950BA60BB70BB3
:100AC0004091E7025091E8026091E9027091EA02D8
:100AD00084179507A607B707B0F28FEF9FEF089529
:100AE000CF93DF93EC018C859D8597FF04C00E9416
:100AF000FB019D878C878C859D85DF91CF91089523
:100B0000FC018485958597FD0BC09FB7F89482E022
:100B10008093E9008091F2009FBF90E001960895D4
:100B20009FB7F89482E08093E9008091F2009FBF24
:100B300090E00895DC01FB0191818081813A31F4DC
:100B40009D7F81E0913009F080E008958132E1F7E6
:100B50009B3029F482811F968C9381E008959A300E
:100B600099F7828150968C93F8CFFC014281FB016A
:100B7000248135814217130611F40C949A0580E004
:100B80000895DC01FB0188E4808389E4818384E4A7
:100B900082831D969C911D979F709F5B93831D96EA
:100BA0008D919C9124E0969587952A95E1F78F7019
:100BB0008F5B848385E00895EF92FF920F931F93DC
:100BC000CF93DF93FB012081213889F523812232E5
:100BD00071F5DC0112964C91248135814217130680
:100BE00031F58C01FC01C385D485F12CE12C2097D3
:100BF00091F04C815D816A817B818E81811180E8D9
:100C00000E9482038F3F980759F0E80EF91E099061
:100C1000D881C02DECCF81E0D8011F968C93C701FD
:100C2000DF91CF911F910F91FF90EF90089590E089
:100C300080E0F6CFCF93DF93CDB7DEB769970FB6DD
:100C4000F894DEBF0FBECDBFFC01DB018C918F5F3E
:100C50008C939E012D5F3F4F8DE0D9011D928A95A7
:100C6000E9F729E0298384E08A8391E09D8383E08A
:100C70008E832A8721E22B879C879D879F8722E28C
:100C8000288B27E02B8B25E02C8B8E8B20E430E00B
:100C9000388F2F8B998F82818B8395858685998B51
:100CA0008A8B838180688D8B49E150E0BE016F5F44
:100CB0007F4F80E00E94820369960FB6F894DEBFF2
:100CC0000FBECDBFDF91CF910895CF9380918B025E
:100CD00081112CC0C1E0C0937E02C0937F0284E8E2
:100CE00092E090938102809380021092830210928E
:100CF000820285E591E090937B0280937A021092C4
:100D00008602109285021092880210928702C09388
:100D10008902C0938A0281EC809384020E9452046B
:100D20006AE772E00E949704C0938B028AE792E020
:100D3000CF910895FC014281FB0124813581421746
:100D4000130611F40C949A0580E00895AF92BF92B7
:100D5000CF92DF92EF92FF920F931F93CF93DF9387
:100D60001F92CDB7DEB77C0169836A01590141E06A
:100D700050E0BE016F5F7F4FFC0183810E94B90389
:100D80008C0197FD0BC0F7018381A501B60180643A
:100D90000E94B903080F191F97FD8C01C8010F901D
:100DA000DF91CF911F910F91FF90EF90DF90CF9047
:100DB000BF90AF900895EF92FF920F931F93CF9340
:100DC000DF93FB012081213871F52381223259F50F
:100DD000DC0112964C91248135814217130619F5D6
:100DE000EC010B851C85F12CE12C0115110589F016
:100DF000F801448155816281738180E80E948203F9
:100E00008F3F980749F0E80EF91ED8010D911C910B
:100E1000ECCF81E08F87C701DF91CF911F910F91B8
:100E2000FF90EF90089590E080E0F6CFCF93DF93AE
:100E3000CDB7DEB769970FB6F894DEBF0FBECDBF52
:100E4000FC01DB018C918F5F8C939E012D5F3F4FE6
:100E50008DE0D9011D928A95E9F729E0298384E084
:100E60008A8391E09D8383E08E832A8721E22B870A
:100E70009C879D879F8722E2288B27E02B8B25E08C
:100E80002C8B8E8B20E430E0388F2F8B998F8281D2
:100E90008B8395858685998B8A8B838180688D8BE2
:100EA00049E150E0BE016F5F7F4F80E00E94820306
:100EB00069960FB6F894DEBF0FBECDBFDF91CF911C
:100EC0000895CF938091670281112CC0C1E0C09337
:100ED0005A02C0935B0280E692E090935D02809399
:100EE0005C0210925F0210925E0289E491E090939E
:100EF0005702809356021092620210926102109281
:100F0000640210926302C0936502C093660281EC92
:100F1000809360020E94520466E572E00E9497048A
:100F2000C093670286E592E0CF910895CF93DF9357
:100F30001F92CDB7DEB791E001C0990F8A95EAF70D
:100F400099830E94610721E030E0AE014F5F5F4F5F
:100F500064E00E94A6060F90DF91CF9108959AE673
:100F6000980F9A3008F051C0863939F0873939F432
:100F70008091F80382608093F80389E817C088396C
:100F800039F48091F80382608093F80387E80EC0FB
:100F9000893909F468C08A3909F467C08B3909F4C2
:100FA00066C08C3909F465C08D3981F39091FA03DC
:100FB0009817F9F09091FB038917D9F09091FC03F1
:100FC0008917B9F09091FD03891799F09091FE036C
:100FD000891779F09091FF03891759F0EAEFF3E050
:100FE00030E020E09191911146C02C503C4FF90126
:100FF00086830E94610728E030E048EF53E062E01A
:101000000E94A60681E090E00895883810F0885884
:10101000CDCFE82FF0E087FF0FC0E058F10921E0C5
:1010200030E001C0220FEA95EAF78091F803822BA5
:101030008093F80380E0BACFE655FE4F849181118A
:1010400009C081E090E09093F7038093F60390E06D
:1010500080E0089587FFAACF9091F8039260909363
:10106000F8038F77A3CF85E3A1CF88E89FCF8AE8E5
:101070009DCF8BE89BCF2F5F3F4F2630310509F086
:10108000B1CFDFCF9AE6980F9A30D8F5863939F08C
:10109000873939F48091F8038D7F8093F80389E8CC
:1010A00017C0883939F48091F8038D7F8093F80355
:1010B00087E80EC0893909F44AC08A3909F449C061
:1010C0008B3909F448C08C3909F447C08D3981F354
:1010D000E4EFF3E096E0882321F02681821301C03B
:1010E0001682915031969111F6CF0E94610728E047
:1010F00030E048EF53E062E00E94A60681E090E015
:101100000895883810F08858E3CFE82FF0E087FF83
:1011100010C0E058F10981E090E001C0880FEA9525
:10112000EAF780959091F80389238093F80380E093
:10113000CFCFE655FE4F8491882389F087FFC8CF33
:101140009091F8039D7F9093F8038F77C1CF85E34B
:10115000BFCF88E8BDCF8AE8BBCF8BE8B9CF90E09E
:1011600080E00895CF93DF9300D000D01F92CDB7D9
:10117000DEB79091410399831A821B828C836D8321
:101180000E94610725E030E0AE014F5F5F4F61E0F4
:101190000E94A6060F900F900F900F900F90DF9176
:1011A000CF9108959091410380958923981731F04C
:1011B0008093410360E080E00C94B2080895909120
:1011C0004103892B981731F08093410360E080E060
:1011D0000C94B20808951092720081E090E0909310
:1011E000D5028093D40280915402909155020396C7
:1011F00090935502809354020895EEECF1E050E094
:1012000040E02FEF30E070E060E0A191B191A817CD
:10121000B90719F46F5F7F4F9A014F5F5F4F4830F6
:10122000510599F72F3F310539F0220F331FF9018E
:10123000E253FE4F118210826230710514F40C9457
:10124000420808950F931F93CF93DF93EEECF1E0E4
:10125000D0E0C0E021913191232B79F4092F182F90
:101260000E94AF07CC0FDD1FC253DE4F18830983E6
:10127000DF91CF911F910F9108952196C830D1052C
:1012800049F7F6CF0895089590E080E00895CF9251
:10129000DF92EF92FF920F931F93CF93DF93CDB71F
:1012A000DEB7A1970FB6F894DEBF0FBECDBF282FD3
:1012B00030E050E040E019A28E010F5D1F4F8AE040
:1012C000C82ED12CE12CF12CCA01B901A70196013D
:1012D0000E944620605DF80162938F01211531055F
:1012E0004105510589F790E080E0309761F0019069
:1012F0000020E9F73197AF01401B510BB80183EE95
:1013000092E00E94DF04A1960FB6F894DEBF0FBEF4
:10131000CDBFDF91CF911F910F91FF90EF90DF90A4
:10132000CF900895CF93DF930E94F504EC0142E043
:1013300050E065E871E083EE92E00E94DF048C0FDC
:101340009D1FDF91CF9108954F925F926F927F9290
:101350008F929F92AF92BF92CF92DF92EF92FF92C5
:101360000F931F93CF93DF93CDB7DEB74DB65EB625
:101370008091E5032DB73EB7281B31090FB6F894CD
:101380003EBF0FBE2DBF8DB79EB701963C0180902A
:101390008803912C8091840390918503D301FC01F3
:1013A0009F01281B390B281539051CF421912D9319
:1013B000F7CF80918903882359F180918003909120
:1013C000810328E097FD09C068E671E00E9477205C
:1013D0006DE270E00E947720262F80918203909129
:1013E000830368E097FD08C068E671E00E947720FB
:1013F0006DE270E00E947720F301E80DF91D90E1A5
:10140000699FB0011124262B2083F40131964F01EE
:101410005301A80CB91CC0909003D0909103E090A8
:101420009203F090930300918C0310918D0320910F
:101430008E0330918F034091540350915503609176
:1014400056037091570380918A0381700E948B012B
:10145000880E991E5301A80CB91CC0909803D09017
:101460009903E0909A03F0909B03009194031091EC
:101470009503209196033091970340915803509122
:10148000590360915A0370915B0380918A0386959A
:1014900081700E948B01880E991E5301A80CB91C03
:1014A000C090A003D090A103E090A203F090A3030A
:1014B00000919C0310919D0320919E0330919F0306
:1014C00040915C0350915D0360915E0370915F03F6
:1014D00080918A0382FB882780F90E948B01880E05
:1014E000991E5301A80CB91CC090A803D090A90361
:1014F000E090AA03F090AB030091A4031091A50320
:101500002091A6033091A70340916003509161039D
:10151000609162037091630380918A0383FB882743
:1015200080F90E948B01880E991E5301A80CB91CEA
:10153000C090B003D090B103E090B203F090B30339
:101540000091AC031091AD032091AE033091AF0335
:101550004091640350916503609166037091670345
:1015600080918A03829581700E948B01880E991E5A
:101570005301A80CB91CC090B803D090B903E090F7
:10158000BA03F090BB030091B4031091B50320910E
:10159000B6033091B703409168035091690360919D
:1015A0006A0370916B0380918A0385FB882780F919
:1015B0000E948B01880E991E5301A80CB91CC09083
:1015C000C003D090C103E090C203F090C303009128
:1015D000BC031091BD032091BE033091BF03409125
:1015E0007003509171036091720370917303809145
:1015F0008B0381700E948B01880E991E5301A80CE9
:10160000B91CC090C803D090C903E090CA03F09001
:10161000CB030091C4031091C5032091C603309100
:10162000C70340916C0350916D0360916E037091FC
:101630006F0380918B03869581700E948B01880EC9
:10164000991E5301A80CB91CC090D003D090D103AF
:10165000E090D203F090D3030091CC031091CD031E
:101660002091CE033091CF034091740350917503C4
:10167000609176037091770380918B0382FB8827BA
:1016800080F90E948B01880E991E5301A80CB91C89
:10169000C090D803D090D903E090DA03F090DB0338
:1016A0000091D4031091D5032091D6033091D70334
:1016B000409178035091790360917A0370917B0394
:1016C00080918B0383FB882780F90E948B01880D12
:1016D000991D5301A80EB91EC090E003D090E103FC
:1016E000E090E203F090E3030091DC031091DD034E
:1016F0002091DE033091DF0340917C0350917D0304
:1017000060917E0370917F0380918B03829581703D
:101710000E948B010E9465064C014091E503809177
:10172000E40350E05A01FFEFAF1ABF0A2DB73EB7EE
:101730002A193B090FB6F8943EBF0FBE2DBF0DB757
:101740001EB70F5F1F4FEDB7FEB78183B301C8010E
:1017500001960E948722F4018381A501B80180646B
:101760000E94B9030FB6F8945EBE0FBE4DBEDF9166
:10177000CF911F910F91FF90EF90DF90CF90BF908E
:10178000AF909F908F907F906F905F904F90089553
:1017900020918903222349F0909381038093800351
:1017A0008091860381110C94A4090895880F991FD4
:1017B000FC01EB5DFE4F0190F081E02D2091E001F6
:1017C0003091E101835E9E4FDC018D919C914091AF
:1017D000DE015091DF01672BE1F42E1B3F0B3093AC
:1017E000E1012093E001481B590B5093DF01409326
:1017F000DE018091E0019091E101009711F5809167
:10180000DE019091DF01009789F48FEF9FEF0C9438
:10181000C80B2E0F3F1F3093E1012093E001840F8E
:10182000951F9093DF018093DE01E3CF8130910516
:1018300019F490E080E0EBCF019681F584EB90E025
:10184000E6CF81309105A1F48091DE019091DF0116
:10185000009719F48AE590E0DACF8130910519F408
:101860008DE290E0D4CF0196C9F487E890E0CFCF25
:101870000196A1F48091DE019091DF01009719F4A7
:101880008EE091E0C4CF8130910519F48BE391E0B3
:10189000BECF019619F481EE90E0B9CF08959091F2
:1018A0008703891700F5E82FE695E695E6952091E0
:1018B000840330918503E20FF32FF11D282F277049
:1018C00081E090E0A0E0B0E004C0880F991FAA1F5B
:1018D000BB1F2A95D2F72081822B808380918603BB
:1018E00081110C94A409089590918703891708F534
:1018F000E82FE695E695E6952091840330918503DF
:10190000E20FF32FF11D282F277081E090E0A0E077
:10191000B0E004C0880F991FAA1FBB1F2A95D2F7F9
:1019200080959081892380838091860381110C9416
:10193000A4090895CF93DF93EC01888199810097E2
:1019400011F00E944121198218821D821C821B8283
:101950001A82DF91CF910895FC01808191810097D7
:1019600011F00C9441210895FC0180819181009730
:1019700011F00C945E1F60E070E0CB010895FC0153
:1019800024813581232B39F421E0FB0180818823D8
:1019900049F020E007C0808191810E94902221E0DF
:1019A000892BB9F7822F08950F931F93CF93DF935D
:1019B000EC0188819981009759F02A813B81261793
:1019C000370730F081E0DF91CF911F910F9108959B
:1019D0008B016F5F7F4F0E94CA21009759F0998356
:1019E00088831B830A832C813D81232B59F7FC01BB
:1019F0001082E8CF80E0E7CFEF92FF920F931F9322
:101A0000CF93DF936115710541F480E0DF91CF91B1
:101A10001F910F91FF90EF90089541155105B1F07E
:101A20007B01EC010C811D81040F151FB8010E9480
:101A3000D40C882351F3288139818C819D81B70191
:101A4000820F931F0E9499221D830C8381E0DECFB9
:101A5000EF92FF920F931F93CF93DF9300D000D0AC
:101A6000CDB7DEB77C01862F4AE08E010F5F1F4F96
:101A7000B80190E00E94851FF80101900020E9F76D
:101A80003197AF01401B510BB801C7010E94FC0CFC
:101A9000811103C0C7010E949A0CC7010F900F90DB
:101AA0000F900F90DF91CF911F910F91FF90EF90CA
:101AB0000895EF92FF920F931F93CF93DF93EC0162
:101AC0007B018A01BA010E94D40C81110BC0CE01A6
:101AD0000E949A0CCE01DF91CF911F910F91FF9040
:101AE000EF9008951D830C83B701888199810E942E
:101AF0009922F0CFEF92FF920F931F93CF93DF9332
:101B0000CDB7DEB762970FB6F894DEBF0FBECDBF7C
:101B10008C01CB01F801118210821382128215828E
:101B200014824AE09E012F5F3F4F7901B9010E9464
:101B3000851FF70101900020E9F73197AF014E1999
:101B40005F09B701C8010E94590D62960FB6F8945B
:101B5000DEBF0FBECDBFDF91CF911F910F91FF90E0
:101B6000EF900895CF93DF93EC01FB018617970761
:101B700049F0608171816115710541F044815581A1
:101B80000E94590DCE01DF91CF9108950E949A0CC9
:101B9000F9CFFC0111821082138212821582148205
:101BA000FB0101900020E9F73197AF01461B570B6D
:101BB0000C94590DCF92DF92EF92FF920F931F93E7
:101BC000CF93DF937C016B018A014617570720F4FE
:101BD0008D2D6A01062F182F67E871E0C7010E945A
:101BE000C90DC0914603D0914703CC16DD0638F5E8
:101BF0000C171D0708F4E801E0914203F09143033C
:101C0000EC0FFD1F1081108260914203709143031D
:101C10006C0D7D1D61157105E1F0FB010190002047
:101C2000E9F73197AF01461B570BC7010E94590DC9
:101C30008091420390914303C80FD91F1883C701B5
:101C4000DF91CF911F910F91FF90EF90DF90CF9098
:101C50000895C7010E949A0CEBCF0C94CF1FEF920E
:101C6000FF920F931F93CF93DF937C01C091520299
:101C7000D09153028091540290915502C80FD91F00
:101C8000CE0101960E942D0E082F10E0CE01029683
:101C90000E942D0E90E0EA94EF2851F428EE33E0F4
:101CA000AC01429FC001439F900D529F900D1124A3
:101CB000809F9001819F300D909F300D1124C901AC
:101CC000330FAA0BBB0B0097A105B10521F481E0EE
:101CD00090E0A0E0B0E08093720290937302A09332
:101CE0007402B09375028BEE98E09093700280932B
:101CF0006F021092C1001092C0001092C2001092A8
:101D0000C3001092C40088E48093C1008CE790E087
:101D10009093510280935002809150029091510211
:101D20008093D1001092760210927702109278027E
:101D3000109279021092710284E089BB1092BF0068
:101D40001092BE0080937200DF91CF911F910F918E
:101D5000FF90EF900895FF920F931F93CF93DF931F
:101D600080E092E0A0E0B0E08093540390935503AC
:101D7000A0935603B09357038091860381110E946C
:101D8000A40980E092E0A0E0B0E080935803909333
:101D90005903A0935A03B0935B038091860381118A
:101DA0000E94A40980E092E0A0E0B0E080935C0390
:101DB00090935D03A0935E03B0935F0380918603CD
:101DC00081110E94A40980E092E0A0E0B0E080933D
:101DD000600390936103A0936203B09363038091C7
:101DE000860381110E94A40980E092E0A0E0B0E0A7
:101DF0008093640390936503A0936603B093670395
:101E00008091860381110E94A40980E092E0A0E005
:101E1000B0E08093680390936903A0936A03B09342
:101E20006B038091860381110E94A40980E092E0F7
:101E3000A0E0B0E080936C0390936D03A0936E03D9
:101E4000B0936F038091860381110E94A40961E021
:101E50008AE00E9497028AE00E9471021092D002EA
:101E60001092CF02C091CF02D091D002C530D105DF
:101E70007CF4FE01EE0FFF1FE35AFE4F62E080810B
:101E80000E9497022196D093D002C093CF02EACF4E
:101E90001092D0021092CF02FF24F394C091CF028F
:101EA000D091D002C530D1050CF041C0CE018C5983
:101EB0009F4F0E942D0E8E01000F111FF801E95552
:101EC000FD4F8F3F41F511821082CE018A569F4F00
:101ED0000E942D0EF801EF54FD4F8F3F01F5118246
:101EE0001082CE0180579E4F0E942D0EF801E554BE
:101EF000FD4F8F3FC1F411821082FE01E653FD4F6A
:101F0000F082FE01EB53FD4FF0822196D093D00278
:101F1000C093CF02C3CF90E091838083D6CF90E06F
:101F200091838083DECF90E091838083E6CF8EE83B
:101F300090E00E942D0E90E001968F3F910551F0A8
:101F40009093010180930001DF91CF911F910F9138
:101F5000FF90089581E090E0F3CFEF92FF920F930E
:101F60001F93CF93DF93CDB7DEB72C970FB6F894BE
:101F7000DEBF0FBECDBF8C01CB017A01181619064A
:101F800014F40E94FD081E141F041CF4C7010E94D3
:101F9000FD08C80180978B3B910508F075C08459F6
:101FA00091090D9790F580E10B3B110521F00C3B59
:101FB000110581F488E00E94D2082C960FB6F8949F
:101FC000DEBF0FBECDBFDF91CF911F910F91FF906C
:101FD000EF900895C8018D5B9109029728F460E0A5
:101FE00080E00E94B208E9CF0F5B110902301105B1
:101FF00020F719820E94610721E030E0AE014F5FB7
:102000005F4F64E00E94A606D8CFC801865A9109A6
:102010008430910528F470E060E00E94D60BCDCFAB
:10202000C801805A9109059708F0E0C0B8016F59BE
:102030007109CE0107960E947A0D68E871E0CE0121
:1020400001960E94C90D4B855C856F817885CE0114
:1020500001960E94FC0C811104C0CE0101960E94E1
:102060009A0CCE0101960E94F504CE0101960E94C1
:10207000AC0CCE0107960E94AC0C64E170E080E0ED
:1020800090E00E94ED0299CFC8018B5D9109849781
:1020900008F0B0C081E0073E110509F48CCF84E060
:1020A000083E110509F487CF82E0093E110509F4C5
:1020B00082CF8EE00E3E110509F4A8C00B3D11053C
:1020C00059F490E080E00E942D0E811176CF10929D
:1020D000E2010E94371171CF0C3D110549F482E3F2
:1020E00090E00E942D0E811168CF1092E301F1CF94
:1020F0000D3D110549F48CE291E00E942D0E8111F5
:102100005CCF1092E401E5CF0E3D110549F48EE558
:1021100091E00E942D0E811150CF1092E501D9CF90
:102120000F3D110549F482EC91E00E942D0E8111C2
:1021300044CF1092E601CDCF003E110549F486E26E
:1021400092E00E942D0E811138CF1092E701C1CF8D
:10215000013E110549F488E592E00E942D0E81119F
:102160002CCF1092E801B5CF023E110549F48AE860
:1021700092E00E942D0E811120CF1092E901A9CF8B
:10218000033E110549F48CEB92E00E942D0E811163
:1021900014CF1092EA019DCF043E110549F48EEE52
:1021A00092E00E942D0E811108CF1092EB0191CF89
:1021B0000C3F110549F480E293E00E942D0E81113D
:1021C000FCCE1092EC0185CF0D3F110549F482E55C
:1021D00093E00E942D0E8111F0CE1092ED0179CF87
:1021E000C801805F91090C9708F0E7CE802F0E940C
:1021F0004208E3CEC80101974F9708F0DECE8CEC81
:10220000800F0F3011059CF78FEF800F0E94740C28
:10221000D4CECF93DF93109272001092D502109219
:10222000D4021092D102E2EEF1E0119281E0EE3E92
:10223000F807D9F7C6EFD1E050E040E070E060E089
:10224000899199910E94AD0FFE01329711821082FF
:1022500082E0C035D80781F787E00E94D20880E18C
:102260000E94D20888E0DF91CF910C94D208E2EE70
:10227000F1E081E0EE3EF80721F081918823C9F377
:1022800008950C940911EF92FF920F931F93CF932F
:10229000DF93CDB7DEB72C970FB6F894DEBF0FBE35
:1022A000CDBF8C01CB017A011816190644F40E94A7
:1022B00022091E141F041CF4C7010E942209C80130
:1022C00080978B3B910508F07EC0845991090D974A
:1022D000E8F50B3B1105A1F48091410384FD03C097
:1022E00080E10E94DF082C960FB6F894DEBF0FBE87
:1022F000CDBFDF91CF911F910F91FF90EF90089587
:102300000C3B110531F48091410383FDECCF88E053
:10231000E8CF6FEF0D3B110521F00E3B110529F4BD
:1023200061E080E00E94B208DECF80E00F3B110543
:1023300021F0003C1105B9F681E00E9496076AE0A1
:1023400070E080E090E00E94ED02CDCFC801865A97
:1023500091098430910528F461E070E00E94D60B69
:10236000C2CFC801805A9109059708F0ACC1B801E5
:102370006F597109CE0107960E947A0D6DE871E0E0
:10238000CE0101960E94C90D4B855C856F817885D1
:10239000CE0101960E94FC0C811104C0CE01019671
:1023A0000E949A0CCE0101960E94F504CE0101967E
:1023B0000E94AC0CCE0107960E94AC0C64E170E068
:1023C00080E090E0C0CFC8018B5D9109859708F04F
:1023D0007EC1073E110531F48091410380FD83CF1A
:1023E00081E07FCF083E110531F48091410382FDE9
:1023F0007ACF84E076CF093E110531F48091410314
:1024000081FD71CF82E06DCF60E0809100010A3ED6
:10241000110509F487CF8091000160E081950B3EA2
:10242000110509F47FCF8EE00E3E110509F45BC162
:102430000B3D1105C9F490E080E00E942D0E90E064
:10244000009751F481E08093E20170E060E090E059
:1024500080E00E94721447CF019709F044CF809129
:10246000E20191E08927EFCF0C3D1105B9F482E339
:1024700090E00E942D0E90E0009741F481E080935F
:10248000E30161E070E082E390E0E3CF019709F0BF
:102490002ACF8091E30191E08927F1CF0D3D11050D
:1024A000B9F48CE291E00E942D0E90E0009741F487
:1024B00081E08093E40162E070E08CE291E0C9CFBA
:1024C000019709F010CF8091E40191E08927F1CFC5
:1024D0000E3D1105B9F48EE591E00E942D0E90E0BD
:1024E000009741F481E08093E50163E070E08EE5C0
:1024F00091E0AFCF019709F0F6CE8091E50191E030
:102500008927F1CF0F3D1105B9F482EC91E00E94CB
:102510002D0E90E0009741F481E08093E60164E0A5
:1025200070E082EC91E095CF019709F0DCCE8091CC
:10253000E60191E08927F1CF003E1105B9F486E26A
:1025400092E00E942D0E90E0009741F481E080938C
:10255000E70165E070E086E292E07BCF019709F049
:10256000C2CE8091E70191E08927F1CF013E1105AC
:10257000B9F488E592E00E942D0E90E0009741F4B6
:1025800081E08093E80166E070E088E592E061CF49
:10259000019709F0A8CE8091E80191E08927F1CF59
:1025A000023E1105B9F48AE892E00E942D0E90E0F7
:1025B000009741F481E08093E90167E070E08AE8E8
:1025C00092E047CF019709F08ECE8091E90191E02A
:1025D0008927F1CF033E1105B9F48CEB92E00E94FC
:1025E0002D0E90E0009741F481E08093EA0168E0CD
:1025F00070E08CEB92E02DCF019709F074CE8091C2
:10260000EA0191E08927F1CF043E1105B9F48EEE7D
:1026100092E00E942D0E90E0009741F481E08093BB
:10262000EB0169E070E08EEE92E013CF019709F0C4
:102630005ACE8091EB0191E08927F1CF0C3F110533
:10264000B9F480E293E00E942D0E90E0009741F4EF
:1026500081E08093EC016AE070E080E293E0F9CEE3
:10266000019709F040CE8091EC0191E08927F1CFEC
:102670000D3F1105B9F482E593E00E942D0E90E024
:10268000009741F481E08093ED016BE070E082E51A
:1026900093E0DFCE019709F026CE8091ED0191E025
:1026A0008927F1CF0F3E110541F482E00E94960781
:1026B00068EC70E080E090E046CEC801805F910950
:1026C0000C9708F010CE802F0E94AF070CCEC801E7
:1026D00001974F9708F007CE8CEC800F0F30110553
:1026E0009CF78FEF800F0E944F0CFDCDEF92FF9271
:1026F0000F931F93CF93DF93EC01E0905202F09081
:1027000053028091540290915502E80EF91EC701C0
:1027100001960E942D0E082F10E0209789F550E0B9
:1027200040E070E060E0C8010E944311E6EFF1E094
:10273000819191910817190741F0892BE1F4CC0F91
:10274000DD1FCA50DE4F1983088380915402909197
:1027500055020396909355028093540281E090E0D5
:102760009093D5028093D402DF91CF911F910F9166
:10277000FF90EF9008952196CD32D105C9F6E5CFAF
:10278000219741F450E040E070E060E0C8010E9411
:10279000AD0FDBCFC70102960E942D0EC82FD0E0EF
:1027A000209711F4CAE0D0E050E040E070E060E033
:1027B000C8010E944311BE01DD0F880B990B0E94D6
:1027C000ED02E0CF0F931F93CF93DF93009152025E
:1027D00010915302C0915402D0915502C00FD11FE5
:1027E000CE010E942D0E9FEF980F9E3F08F443C02C
:1027F0008091F4019091F50101969093F5018093F9
:10280000F4012091F2013091F30121153105C1F459
:102810008091F0019091F1010817190721F0909330
:1028200053028093520281E090E09093D50280930E
:10283000D40283E090E0909355028093540216C036
:10284000821793072CF31092D1021092D5021092A6
:10285000D4028091D2029091D302019739F4E09191
:10286000EE01F091EF01EE51FE4F1082DF91CF911A
:102870001F910F910895282F30E0813041F490E0AE
:1028800080E0DF91CF911F910F910C94761322304D
:10289000310519F481E090E0F4CF82E090E023303C
:1028A000310579F390E080E02430310529F02530BE
:1028B000310541F481E090E0DF91CF911F910F91BC
:1028C0000C942F0E2630310589F6CE0101960E9418
:1028D0002D0EE82FF0E0EE0FFF1FE35DFE4F80812D
:1028E00091819DCF0F931F93CF939093F10180938C
:1028F000F00190935302809352027093EF01609322
:10290000EE016E517E4FFB0180818823D1F18091D1
:10291000D10281110E940911E091EE01F091EF01C5
:10292000EE51FE4FC1E0C0831092D5021092D40246
:1029300083E090E0909355028093540200915202FC
:1029400010915302C8010E942D0E90E09093D30283
:102950008093D2028F3F9105C9F0C80101960E9471
:102960002D0E90E09093F3018093F2011092F50107
:102970001092F401C093D102CF911F910F910C944A
:10298000E213CF911F910F910C940911CF911F91D8
:102990000F9108951F920F920FB60F9211242F934B
:1029A0003F938F939F93AF93BF938091DF0290915A
:1029B000E002A091E102B091E2023091D80223E05E
:1029C000230F2D3758F50196A11DB11D2093D80274
:1029D0008093DF029093E002A093E102B093E202C1
:1029E0008091D9029091DA02A091DB02B091DC02D1
:1029F0000196A11DB11D8093D9029093DA02A09394
:102A0000DB02B093DC02BF91AF919F918F913F9118
:102A10002F910F900FBE0F901F90189526E8230F4F
:102A20000296A11DB11DD2CF1F920F920FB60F9229
:102A300011248F939F938091E1009091E100937F07
:102A40009093E10083FF0FC01092E90091E0909312
:102A5000EB001092EC0092E39093ED001092DE02F6
:102A600098E09093F00082FF22C093E09093E900F9
:102A70009091F200992319F09AE39093E8009091D5
:102A8000A402992341F09091A40291509093A40242
:102A9000911101C05D9A9091DD02992341F09091CE
:102AA000DD0291509093DD02911101C0289A84FFBC
:102AB00018C08091E2008E7E81608093E200809158
:102AC000E1008F7E8093E1008091A5028E7E80617F
:102AD0008093A5029F918F910F900FBE0F901F9032
:102AE000189580FFF7CF8091E2008E7E8061809301
:102AF000E2008091E1008E7E8093E1008091A5024A
:102B00008E7E8160E5CF1F920F920FB60F92112437
:102B1000CF92DF92EF92FF920F931F932F933F93E9
:102B20004F935F936F937F938F939F93AF93BF93D5
:102B3000EF93FF93CF93DF93CDB7DEB76C97DEBFF4
:102B4000CDBF1092E9008091E80083FF2FC089E09B
:102B5000FE017596EE2EDF2E815029F09091F10046
:102B600090833196F9CF84E68093DD0282EF8093E3
:102B7000E8008D8987FF39C09091E80090FFFCCF75
:102B8000982F907609F033C19E894F89588D2F89EF
:102B9000F88C911131C0803861F58091A602809344
:102BA000F1001092F1008EEF8093E8006C960FB662
:102BB000F894DEBF0FBECDBFDF91CF91FF91EF91B3
:102BC000BF91AF919F918F917F916F915F914F9145
:102BD0003F912F911F910F91FF90EF90DF90CF9039
:102BE0000F900FBE0F901F9018959EEF9093E800E6
:102BF000C7CF1092F100D5CF913059F48111D3CFC6
:102C00004130510581F68091A6028D7F8093A60206
:102C1000CACF933049F48111C6CF4130510519F61E
:102C20008091A6028260F2CF953041F48091E80055
:102C300080FFFCCF20682093E300B5CF963009F0E9
:102C4000A8C00B8D1C8D22E01092E9001092A20208
:102C50001092A102F2122EC01092A00210929F02B6
:102C60000E9466041F8299E09983FA8291E09E8314
:102C700090EA98879AEF99872091A1023091A20259
:102C8000275F3F4F3C832B838D831092E900109286
:102C9000A2021092A1021093A00200939F0249E0A9
:102CA00050E0BE016F5F7F4F80E00E9482030E9470
:102CB000660479CF1093A00200939F020E945204F1
:102CC000DC0112960D911C910115110509F457C1F3
:102CD000D801ED91FC910480F581E02D6E2D7D2DC4
:102CE000C8010995009709F045C1F80100851185D3
:102CF000EBCFF3E0FF120EC08F89882309F440C0A8
:102D0000823061F440E862E180E191E00E944F038B
:102D1000811149CF81E28093EB0048CF813029F4C3
:102D200040E86BE084E091E0F1CF833099F70E94B6
:102D30005204DC011296ED90FC908E010F5F1F4F44
:102D40006801E114F10479F0D701ED91FC9106805E
:102D5000F781E02DB801C7010995080F111DF70192
:102D6000E084F184EECFD8011C92F601019000209E
:102D7000E9F73197BF016C197D0940E0C601C6CF64
:102D80006EEE70E0FB01449150E080E80E94820307
:102D90000ACF973009F4BECF983021F481E08093B8
:102DA000F10001CF993009F0FECE837009F0B2CF67
:102DB000E3E0F1E081E031E096E32191222371F03C
:102DC0008093E9003093EB00DF0111972C91209361
:102DD000EC009093ED008F5F873079F78EE780935A
:102DE000EA001092EA008F898093DE02DCCE8B8DA0
:102DF0009C8D1092E9001092A2021092A102909371
:102E0000A00280939F02898D81119AC08E899D892D
:102E1000913A49F4813209F07DCF47E050E06DE00E
:102E200071E080E0B3CF913209F074CF833269F45E
:102E30008F89988DB0E0A0E08093090190930A01FA
:102E4000A0930B01B0930C01AECE8032A9F4809117
:102E5000E80082FFFCCF88E0EDE0F1E0815029F04E
:102E60009091F10090833196F9CF84E68093DD0252
:102E70008BEF8093E80097CE823209F094CE8F8951
:102E800080931401EEEFFFE7859194918B3F9C4D69
:102E900051F1E0E0F8E080910D0190910E01A091D8
:102EA0000F01B0911001803B9440A105B105F1F4F0
:102EB0008091140180FD1AC0EE3F8AE0F80789F581
:102EC00087E797E791838083809160008093A302D6
:102ED00088E19BE00FB6F894A895809360000FBE40
:102EE0009093600060CEEEEFFAE0D5CF80819181C3
:102EF0008737974709F057CEA89580916000886181
:102F0000809360008091A30280936000EE3F2AE0EE
:102F1000F20789F08091FE0A9091FF0A91838083E5
:102F200042CE808191818737980751F29093FF0AB2
:102F30008093FE0AC5CF1092FF0A1092FE0A33CE8C
:102F40000E945204DC0112960D911C91011511058D
:102F500009F4E0CED801ED91FC910190F081E02DD3
:102F60006E2D7D2DC801099581111DCEF8010085BA
:102F70001185ECCF181619060CF415CECBCEF1E066
:102F8000FF12B7CE62EF70E0FDCE1F920F920FB628
:102F90000F9211242F933F934F935F936F937F93DF
:102FA0008F939F93AF93BF93EF93FF93809176029C
:102FB00090917702A0917802B09179020196A11DBB
:102FC000B11D8093760290937702A0937802B0931C
:102FD00079028091760290917702A0917802B09167
:102FE0007902409172025091730260917402709163
:102FF000750284179507A607B70710F18091710233
:1030000081111EC081E080937102809176029091BF
:103010007702A0917802B0917902841B950BA60BE0
:10302000B70B8093760290937702A0937802B093C7
:103030007902E0916F02F09170020995109271028D
:10304000FF91EF91BF91AF919F918F917F916F9180
:103050005F914F913F912F910F900FBE0F901F9056
:103060001895FC01A385B485109771F47487638764
:1030700085859685DB0114962D913C91820F931FD7
:10308000968785870895DC018D919C911197009713
:10309000D1F76D937C93ECCFCF92DF92EF92FF92BA
:1030A0000F931F93CF93DF93CDB7DEB7C659D109E6
:1030B0000FB6F894DEBF0FBECDBF1092E60210929D
:1030C000E50288EE93E0A0E0B0E08093E702909301
:1030D000E802A093E902B093EA028BE691E09093B4
:1030E000E4028093E3028FEF9FEF9093F0028093CE
:1030F000EF021092410380913903811113C01092A5
:103100003403109233038AE292E090933603809363
:10311000350385E490E0909338038093370381E092
:10312000809339030E94610763E373E00E943118C2
:1031300010928503109284031092880310928C03DE
:1031400010928D0310928E0310928F038FEF93E0F5
:10315000A0E0B0E08093900390939103A09392033A
:10316000B0939303109294031092950310929603D8
:10317000109297038093980390939903A0939A03D6
:10318000B0939B0310929C0310929D0310929E0398
:1031900010929F038093A0039093A103A093A20396
:1031A000B093A3031092A4031092A5031092A60358
:1031B0001092A7038093A8039093A903A093AA0356
:1031C000B093AB031092AC031092AD031092AE0318
:1031D0001092AF038093B0039093B103A093B20316
:1031E000B093B3031092B4031092B5031092B603D8
:1031F0001092B7038093B8039093B903A093BA03D6
:10320000B093BB031092BC031092BD031092BE0397
:103210001092BF038093C0039093C103A093C20395
:10322000B093C3031092C4031092C5031092C60357
:103230001092C7038093C8039093C903A093CA0355
:10324000B093CB031092CC031092CD031092CE0317
:103250001092CF038093D0039093D103A093D20315
:10326000B093D3031092D4031092D5031092D603D7
:103270001092D7038093D8039093D903A093DA03D5
:10328000B093DB031092DC031092DD031092DE0397
:103290001092DF038093E0039093E103A093E20395
:1032A000B093E30353E05093E40330E23093870399
:1032B00022E0209389038FE380938A038FE1809338
:1032C0008B0345E0498391E09A8389E08B83A4E0F6
:1032D000AC83F1EAFD839E8365E86F835887498755
:1032E0008A8759E15B879C8759E25D873E8775E154
:1032F0007F87188A15E2198B9A8B65E76B8B9C8BFD
:1033000055E95D8B3E8B35E53F8B188EB5E6B98F61
:103310001A8E31E83B8F2C8F4D8F9E8F8F8FE9E374
:10332000CE2EC8A279A31AA21BA307E0D02EDCA23E
:10333000E5E3EDA31EA206E4E02EEFA20BE3F02EE0
:10334000F8A699A7BAA704E10BA76CA7ADA75EA73B
:103350009FA738AB29AB8AABCBAA7CAB1DAA1EAB0F
:10336000DFAAE8AF19AEEAAEFBAE9CAFBDAF0EAFC1
:103370006FAF2196AFAF219722965FAF229723962A
:103380009FAF239724963FAF249725962FAF25977D
:1033900026968FAF269727969FAF279728967FAFC1
:1033A000289729961FAE2997B7E22A96BFAF2A978A
:1033B0009FEF2B969FAF2B972C969FAF2C972D9618
:1033C0001FAE2D972E961FAE2E972F966FAF2F976D
:1033D000A0E16096AFAF609761965FAF619716E02E
:1033E00062961FAF62976396FFAF639764961FAEB6
:1033F000649765968FAF659710E366961FAF6697E3
:1034000067968FAF679711E368961FAF68976996C5
:103410008FAF699712E36A961FAF6A976B968FAF6B
:103420006B9713E36C961FAF6C976D968FAF6D978C
:1034300014E36E961FAF6E976F968FAF6F97A0963F
:10344000EFAFA097A1963FAFA197A2962FAFA297FB
:10345000E0ECA396EFAFA397A4964FAFA497A596E1
:103460002FAFA597A6967FAFA697A7961FAEA79753
:10347000A896BFAFA897A9969FAFA997AA969FAF06
:10348000AA97AB961FAEAB97AC961FAEAC97AD9616
:103490006FAFAD97AE96AFAFAE97AF965FAFAF974A
:1034A000E0964FAFE097E196FFAFE197E2961FAE4F
:1034B000E297E3968FAFE3979AEBE4969FAFE4979A
:1034C000E5968FAFE5979BEBE6969FAFE697E7967D
:1034D0008FAFE79794ECE8969FAFE897E9968FAFA8
:1034E000E99795ECEA969FAFEA97EB968FAFEB974B
:1034F00088ECEC968FAFEC97ED963FAFED97EE969C
:103500002FAFEE97EF96EFAFEF97C158DF4FE883FD
:10351000CF57D0408FE790E00E94A5207C018FE735
:10352000FE013196D70101900D928A95E1F787E06F
:1035300090E00E94A5208C01DC0111961C921E9245
:103540001396FC92EE9212978FE790E015969C935B
:103550008E93149716961C920E946506FC01A38513
:10356000B485109709F0A3C01487038785859685D5
:10357000D80114962D913C91820F931F96878587D1
:1035800090918703892F869586958695977009F087
:1035900096C08093880310918803812F90E0009754
:1035A00011F481E090E00E94A52090938503809320
:1035B000840381E090918903911101C080E01A5E3B
:1035C000810F8093E50310925403109255031092DB
:1035D00056031092570310925803109259031092F9
:1035E0005A0310925B0310925C0310925D031092D9
:1035F0005E0310925F0310926003109261031092B9
:103600006203109263031092640310926503109298
:103610006603109267031092680310926903109278
:103620006A0310926B0310926C0310926D03109258
:103630006E0310926F031092700310927103109238
:103640007203109273031092740310927503109218
:1036500076031092770310927803109279031092F8
:103660007A0310927B0310927C0310927D031092D8
:103670007E0310927F038FEF9FEF909381038093DF
:103680008003909383038093820390E080E02091F5
:10369000880328171906A9F0A4F0E0918403F0919B
:1036A0008503E80FF91F10820196F1CFDC018D919F
:1036B0009C9111970097D1F70D931C9357CF8F5F73
:1036C00068CF62E971E08EE493E00E94C90D6AE977
:1036D00071E088E493E00E94C90D67E871E082E43C
:1036E00093E00E94C90D1092F7031092F6038DE744
:1036F00091E09093F5038093F4038091EC038111A2
:1037000013C01092E7031092E6038FE692E09093C5
:10371000E9038093E8038FE290E09093EB038093BA
:10372000EA0381E08093EC030E94610766EE73E098
:103730000E94311880910604811113C01092010477
:10374000109200048EE992E09093030480930204A7
:103750008FE190E0909305048093040481E08093CE
:1037600006040E94610760E074E0CA56DF4F0FB69E
:10377000F894DEBF0FBECDBFDF91CF911F910F91A7
:10378000FF90EF90DF90CF900C943118CF93DF93A0
:10379000CDB7DEB72C970FB6F894DEBF0FBECDBF06
:1037A000789484B5826084BD84B5816084BD85B51C
:1037B000826085BD85B5816085BD80916E00816028
:1037C00080936E00109281008091810082608093CE
:1037D00081008091810081608093810080918000D0
:1037E000816080938000809191008260809391003D
:1037F0008091910081608093910080919000816020
:10380000809390008091C10084608093C10080917A
:10381000C10082608093C1008091C100816080936B
:10382000C1008091C30081608093C3008091C0007B
:1038300082608093C0008091C20081608093C2004A
:1038400080917A00846080937A0080917A0082600F
:1038500080937A0080917A00816080937A008091D1
:103860007A00806880937A001092DE021092A6029D
:103870001092A5028091D70081608093D70080EAE2
:103880008093D80089B5806189BD89B5826089BD82
:1038900009B400FEFDCF61E070E080E090E00E949E
:1038A000ED028091D8008F7C80618093D800809158
:1038B000E000807F8093E0008091E1008E7E809325
:1038C000E1008DE08093E200559A209A61E08EE15C
:1038D0000E9497028EE10E94710261E081E10E94E4
:1038E000970281E10E9471028FEF9FEF9093F002A7
:1038F0008093EF020E94AB0E81E0809386030E94CA
:10390000A4091092940310929503109296031092BA
:1039100097038FEF93E0A0E0B0E08093980390933B
:103920009903A0939A03B0939B0310928C03109277
:103930008D0310928E0310928F03809390039093C7
:103940009103A0939203B093930364E670E080E048
:1039500090E00E94ED0225E0A22E30E0C32E30E080
:10396000D32E83EE92E00E948005892B09F4F8C1E2
:1039700067E871E0CE0101960E94C90D0E943005F2
:1039800097FD0FC08B33910561F08F83188641E05E
:1039900050E0BE01695F7F4FCE0101960E94FC0C92
:1039A000EDCF8091420390914303009709F440C109
:1039B00069817A816115710509F438C14091440328
:1039C000509145032D813E814217530708F42EC1C3
:1039D0000E9499228D819E81909347038093460394
:1039E0001E821D82CE0101960E94AC0C47E050E081
:1039F00070E060E0CE0101960E94DA0D6CE971E0A2
:103A0000CE0101960E94BF0C182FCE0101960E9494
:103A1000AC0C112309F423C147E050E064E070E0EE
:103A2000CE0101960E94DA0DCE0101960E94B40CDF
:103A30002B017093D7026093D602CE0101960E94AB
:103A4000AC0C4AE050E067E070E0CE0101960E94C5
:103A5000DA0DCE0101960E94B40C709316016093AA
:103A60001501CE0101960E94AC0C8AE2480E511C51
:103A7000C2010E942D0E182FB201CE0107960E949E
:103A80007A0D1A8219821C821B821E821D82BE013F
:103A9000695F7F4FCE0101960E94B20D612FCE016A
:103AA00001960E94280D0E949209CE0101960E9463
:103AB000AC0CCE0107960E94AC0C60911501709180
:103AC0001601072E000C880B990B0E94ED0210E0E6
:103AD00000E0E090D602F090D702E00EF11EC701A0
:103AE0000E942D0EB82EB701CE0107960E947A0DC6
:103AF0001A8219821C821B821E821D82BE01695F8E
:103B00007F4FCE0101960E94B20D6B2DCE01019622
:103B10000E94280D0E949209CE0101960E94AC0CD1
:103B2000CE0107960E94AC0C6091150170911601B0
:103B3000072E000C880B990B0E94ED02E090D60234
:103B4000F090D702E00EF11EA2E3EA0EF11CC701CD
:103B50000E942D0EB82EB701CE0107960E947A0D55
:103B60001A8219821C821B821E821D82BE01695F1D
:103B70007F4FCE0101960E94B20D6B2DCE010196B2
:103B80000E94280D0E949209CE0101960E94AC0C61
:103B9000CE0107960E94AC0C609115017091160140
:103BA000072E000C880B990B0E94ED02E090D602C4
:103BB000F090D702E00EF11EB4EDEB1ABEEFFB0A57
:103BC000C7010E942D0EB82EB701CE0107960E94A4
:103BD0007A0D1A8219821C821B821E821D82BE01EE
:103BE000695F7F4FCE0101960E94B20D6B2DCE0111
:103BF00001960E94280D0E949209CE0101960E9412
:103C0000AC0CCE0107960E94AC0C6091150170912E
:103C10001601072E000C880B990B0E94ED020F5F16
:103C20001F4F0530110509F054CF9BCE0E94412152
:103C300089819A8190934303809342038B819C8175
:103C400090934503809344038D819E819093470315
:103C5000809346031A8219821C821B82C1CE45E0E2
:103C600050E070E060E0CE0101960E94DA0D64EA57
:103C700071E0CE0101960E94BF0C182FCE01019673
:103C80000E94AC0C8EE493E011110AC06AEA71E064
:103C900082E493E00E94BF0C8823A1F088E493E0C3
:103CA0000E94F5048091150190911601A89EB00123
:103CB000A99E700D1124072E000C880B990B0E94F1
:103CC000ED024FCE62EB71E082E493E00E94BF0C04
:103CD000882339F08BE893E00E942D0E0E9447095B
:103CE000E1CF6BEB71E082E493E00E94BF0C88238C
:103CF00019F084E893E0F0CF65EC71E082E493E0A2
:103D00000E94BF0C882319F00E94AB0E2ACE43E01C
:103D100050E070E060E0CE0101960E94DA0DCE0125
:103D200001960E94B40C2B01CE0101960E94AC0CAE
:103D3000409146035091470363E070E0CE01019645
:103D40000E94DA0DCE0101960E94B40C162FCE010E
:103D500001960E94AC0C612FC2010E94D71F01CEB8
:103D60002E981092D0021092CF02E090CF02F090E5
:103D7000D00285E0E816F1040CF064C08701000F62
:103D8000111FF801E35AFE4F208131813327F901D9
:103D9000E557FE4F8491F901E459FE4FB490F901C3
:103DA000E35BFE4F949030E020E0992099F0811180
:103DB0000E942502E92DF0E0EE0FFF1FED5DFE4FA2
:103DC000A591B491EC91BE2291E080E009F490E0DD
:103DD000292F382FF701E653FD4F822F8170808302
:103DE000F701EB53FD4F90818917F9F0F801E55485
:103DF000FD4F40815181F801EF54FD4F6081718189
:103E0000F801E955FD4F80819181232BC1F40E9477
:103E100043118091CF029091D002FC01EB53FD4FF2
:103E200086539D4FDC018C9180838091CF029091CD
:103E3000D00201969093D0028093CF0296CF0E9439
:103E4000AD0FE7CF2E9A65E070E080E090E00E9431
:103E5000ED028091D4029091D502019781F41092E5
:103E6000D5021092D4028091D2029091D302009791
:103E7000B1F48091D102882379F00E94E21365E0C9
:103E800070E080E090E00E94ED02C114D10409F4DA
:103E900068CD0E94000065CD0E940911F0CF019706
:103EA00071F7EBCF82E493E00E94AC0C88E493E0DE
:103EB0000E94AC0C8EE493E00C94AC0C1F93FC01BC
:103EC00099278827BC01E89411911032E9F3193041
:103ED00010F01E30C8F31B3251F01D3249F46894C3
:103EE00006C00E94901F610F711D811D911D1191CF
:103EF00010531A30B0F33EF490958095709561950B
:103F00007F4F8F4F9F4F1F910895BB274A3031F449
:103F1000992322F4BDE2909581959F4F0C94A61FA2
:103F2000592F482F372F262F660F771F881F991F6D
:103F3000660F771F881F991F620F731F841F951FBD
:103F4000660F771F881F991F0895BB27FB01552710
:103F5000AA27880F991FAA1FA41710F0A41B8395E6
:103F60005051B9F7A05DAA3308F0A95DA19300975D
:103F700079F7B111B1931192CB010C94BF1FDC0101
:103F8000FC01672F71917723E1F7329704C07C9190
:103F90006D9370836291AE17BF07C8F30895F999C6
:103FA000FECF92BD81BDF89A992780B50895262F3E
:103FB000F999FECF1FBA92BD81BD20BD0FB6F8940E
:103FC000FA9AF99A0FBE01960895052E97FB1EF4F2
:103FD00000940E94FC1F57FD07D00E94462007FC5A
:103FE00003D04EF40C94FC1F5095409530952195CC
:103FF0003F4F4F4F5F4F0895909580957095619515
:104000007F4F8F4F9F4F08950E946820A59F900D6E
:10401000B49F900DA49F800D911D112408952F929F
:104020003F924F925F926F927F928F929F92AF9248
:10403000BF92CF92DF92EF92FF920F931F93CF9395
:10404000DF93CDB7DEB7CA1BDB0B0FB6F894DEBF2C
:104050000FBECDBF09942A88398848885F846E8452
:104060007D848C849B84AA84B984C884DF80EE809C
:10407000FD800C811B81AA81B981CE0FD11D0FB6A5
:10408000F894DEBF0FBECDBFED010895A1E21A2E58
:10409000AA1BBB1BFD010DC0AA1FBB1FEE1FFF1FEC
:1040A000A217B307E407F50720F0A21BB30BE40B3C
:1040B000F50B661F771F881F991F1A9469F7609583
:1040C0007095809590959B01AC01BD01CF0108953D
:1040D000A29FB001B39FC001A39F700D811D112449
:1040E000911DB29F700D811D1124911D089597FBA4
:1040F000072E16F4009407D077FD09D00E94912076
:1041000007FC05D03EF4909581959F4F08957095DA
:1041100061957F4F0895EE0FFF1F0590F491E02DFC
:104120000994AA1BBB1B51E107C0AA1FBB1FA617FE
:10413000B70710F0A61BB70B881F991F5A95A9F750
:1041400080959095BC01CD0108950F931F93CF9357
:10415000DF938230910510F482E090E0E09110044A
:10416000F091110430E020E0B0E0A0E0309799F445
:104170002115310509F44AC0281B390B24303105BB
:10418000D8F58A819B816115710589F1FB019383C3
:104190008283FE0111C04081518102811381481741
:1041A0005907E0F04817590799F4109761F01296F3
:1041B0000C93129713961C933296CF01DF91CF91F7
:1041C0001F910F9108950093100410931104F4CFE0
:1041D0002115310551F04217530738F0A901DB01D1
:1041E0009A01BD01DF01F801C1CFEF01F9CF909332
:1041F000110480931004CDCFFE01E20FF31F8193D1
:1042000091932250310939832883D7CF20910E040E
:1042100030910F04232B41F42091190130911A01A0
:1042200030930F0420930E04209117013091180150
:104230002115310541F42DB73EB740911B01509136
:104240001C01241B350BE0910E04F0910F04E217C2
:10425000F307A0F42E1B3F0B2817390778F0AC01A9
:104260004E5F5F4F2417350748F04E0F5F1F509386
:104270000F0440930E04819391939FCFF0E0E0E010
:104280009CCFCF93DF930097E9F0FC013297138224
:104290001282A0911004B0911104ED0130E020E0F1
:1042A0001097A1F420813181820F931F20910E0479
:1042B00030910F042817390709F061C0F0930F04FB
:1042C000E0930E04DF91CF910895EA01CE17DF0746
:1042D000E8F54A815B819E0141155105B1F7E9017D
:1042E000FB83EA8349915991C40FD51FEC17FD0751
:1042F00061F4808191810296840F951FE901998371
:104300008883828193819B838A83F0E0E0E0129628
:104310008D919C9113970097B9F52D913C91119730
:10432000CD010296820F931F20910E0430910F044D
:104330002817390739F6309751F510921104109269
:104340001004B0930F04A0930E04BCCFD383C28398
:1043500040815181840F951FC817D90761F44E5FC2
:104360005F4F88819981480F591F518340838A810B
:104370009B81938382832115310509F0B0CFF0939F
:104380001104E09310049ECFFD01DC01C0CF138225
:104390001282D7CFB0E0A0E0E0EDF1E20C94112062
:1043A0008C01009751F4CB010E94A5208C01C8011B
:1043B000CDB7DEB7E0E10C942D20FC01E60FF71F2E
:1043C0009C0122503109E217F30708F49DC0D9017E
:1043D000CD91DC911197C617D70798F0C530D1055C
:1043E00030F3CE0104978617970708F3C61BD70B47
:1043F0002297C193D1936D937C93CF010E94412169
:10440000D6CF5B01AC1ABD0A4C018C0E9D1EA0914B
:104410001004B0911104512C412CF12CE12C109777
:1044200031F580910E0490910F048815990509F0DB
:104430005CC04616570608F058C08091170190914D
:104440001801009741F48DB79EB740911B01509120
:104450001C01841B950BE817F90708F055C0F09371
:104460000F04E0930E04F90171836083A0CF8D9156
:104470009C91119712966C90129713967C901397BB
:10448000A815B90559F56C0142E0C40ED11CCA1437
:10449000DB0420F1AC014A195B09DA011296159789
:1044A00080F06282738251834083D9016D937C9343
:1044B000E114F10471F0D7011396FC93EE93129777
:1044C00076CF22968C0F9D1FF90191838083F30193
:1044D000EFCFF0931104E093100469CF481659060A
:1044E00008F42C017D01D3019ACFCB010E94A520B5
:1044F0007C01009749F0AE01B8010E948722C801F3
:104500000E944121870153CF10E000E050CFFB0112
:10451000DC0102C001900D9241505040D8F708953F
:10452000FB01DC018D91019080190110D9F3990BE9
:104530000895FB01DC0101900D920020E1F7089540
:1045400011E0C0E6D1E004C0FE010E948B2021965C
:0A455000C136D107C9F7F894FFCF78
:10455A00010000C18081000000FFFFFFFF00E100B1
:10456A000000000000640000001204800001000046
:10457A0000FFFF00000000FFFF0000010000003202
:10458A00002C015E01C201260258028A02BC02EE18
:10459A000220035203000000009A061607DB06C138
:1045AA000500000000B5051A06DC05C1050800076C
:1045BA000006000500040000000000FE04DF041FDE
:1045CA000514058005240570050000000043094212
:1045DA0009440920030D0A00687562520068756271
:1045EA0050006D682D6265746100390072656164FE
:1045FA003130300072656164790076657273696F73
:10460A006E006B6579626F617264006469726563DA
:0E461A0074696F6E00636F6D706C657465007F
:00000001FF
